 jncrypto

 Timestamp is 6a16388f (Tue May 26 20:19:27 2026)

 Preferred load address is 10000000

 Start         Length     Name                   Class
 0001:00000000 000043fdH .text$mn                CODE
 0002:00000000 000000ccH .idata$5                DATA
 0002:000000cc 00000008H .00cfg                  DATA
 0002:000000d4 00000004H .CRT$XCA                DATA
 0002:000000d8 00000004H .CRT$XCZ                DATA
 0002:000000dc 00000004H .CRT$XIA                DATA
 0002:000000e0 00000004H .CRT$XIZ                DATA
 0002:000000e4 00000004H .CRT$XPA                DATA
 0002:000000e8 00000004H .CRT$XPZ                DATA
 0002:000000ec 00000004H .CRT$XTA                DATA
 0002:000000f0 00000008H .CRT$XTZ                DATA
 0002:000000f4 00000000H .gfids$y                DATA
 0002:000000f8 00000d88H .rdata                  DATA
 0002:00000e80 00000000H .rdata$CastGuardVftablesA DATA
 0002:00000e80 00000000H .rdata$CastGuardVftablesC DATA
 0002:00000e80 00000004H .rdata$sxdata           DATA
 0002:00000e84 0000005cH .rdata$voltmd           DATA
 0002:00000ee0 000002f4H .rdata$zzzdbg           DATA
 0002:000011d4 00000004H .rtc$IAA                DATA
 0002:000011d8 00000004H .rtc$IZZ                DATA
 0002:000011dc 00000004H .rtc$TAA                DATA
 0002:000011e0 00000008H .rtc$TZZ                DATA
 0002:000011e8 00000088H .xdata$x                DATA
 0002:00001270 000008a4H .edata                  DATA
 0002:00001b14 00000078H .idata$2                DATA
 0002:00001b8c 00000014H .idata$3                DATA
 0002:00001ba0 000000ccH .idata$4                DATA
 0002:00001c6c 000003feH .idata$6                DATA
 0003:00000000 00000018H .data                   DATA
 0003:00000018 000004e4H .bss                    DATA
 0004:00000000 00000060H .rsrc$01                DATA
 0004:00000060 00000370H .rsrc$02                DATA

  Address         Publics by Value              Rva+Base       Lib:Object

 0000:00000000       ___AbsoluteZero            00000000     <absolute>
 0000:00000000       ___arm64x_extra_rfe_table  00000000     <absolute>
 0000:00000000       ___arm64x_extra_rfe_table_size 00000000     <absolute>
 0000:00000000       ___arm64x_native_entrypoint 00000000     <absolute>
 0000:00000000       ___arm64x_redirection_metadata 00000000     <absolute>
 0000:00000000       ___arm64x_redirection_metadata_count 00000000     <absolute>
 0000:00000000       ___dynamic_value_reloc_table 00000000     <absolute>
 0000:00000000       ___enclave_config          00000000     <absolute>
 0000:00000000       ___guard_check_icall_a64n_fptr 00000000     <absolute>
 0000:00000000       ___guard_eh_cont_count     00000000     <absolute>
 0000:00000000       ___guard_eh_cont_table     00000000     <absolute>
 0000:00000000       ___guard_fids_count        00000000     <absolute>
 0000:00000000       ___guard_fids_table        00000000     <absolute>
 0000:00000000       ___guard_iat_count         00000000     <absolute>
 0000:00000000       ___guard_iat_table         00000000     <absolute>
 0000:00000000       ___guard_longjmp_count     00000000     <absolute>
 0000:00000000       ___guard_longjmp_table     00000000     <absolute>
 0000:00000000       ___hybrid_auxiliary_iat    00000000     <absolute>
 0000:00000000       ___hybrid_auxiliary_iat_copy 00000000     <absolute>
 0000:00000000       ___hybrid_code_map         00000000     <absolute>
 0000:00000000       ___hybrid_code_map_count   00000000     <absolute>
 0000:00000000       ___x64_code_ranges_to_entry_points 00000000     <absolute>
 0000:00000000       ___x64_code_ranges_to_entry_points_count 00000000     <absolute>
 0000:00000001       ___safe_se_handler_count   00000001     <absolute>
 0000:00000100       ___guard_flags             00000100     <absolute>
 0000:00000000       ___ImageBase               10000000     <linker-defined>
 0001:00000171       _JNI_OnUnload@8            10001171 f   NativeCrypto.obj
 0001:00000210       _Java_jdk_crypto_jniprovider_NativeCrypto_CBCFinalEncrypt@36 10001210 f   NativeCrypto.obj
 0001:00000334       _Java_jdk_crypto_jniprovider_NativeCrypto_CBCInit@40 10001334 f   NativeCrypto.obj
 0001:00000414       _Java_jdk_crypto_jniprovider_NativeCrypto_CBCUpdate@36 10001414 f   NativeCrypto.obj
 0001:000004d7       _Java_jdk_crypto_jniprovider_NativeCrypto_CreateContext@8 100014d7 f   NativeCrypto.obj
 0001:000004f1       _Java_jdk_crypto_jniprovider_NativeCrypto_DestroyContext@16 100014f1 f   NativeCrypto.obj
 0001:0000050d       _Java_jdk_crypto_jniprovider_NativeCrypto_DigestComputeAndReset@40 1000150d f   NativeCrypto.obj
 0001:00000624       _Java_jdk_crypto_jniprovider_NativeCrypto_DigestCreateContext@20 10001624 f   NativeCrypto.obj
 0001:0000074c       _Java_jdk_crypto_jniprovider_NativeCrypto_DigestDestroyContext@16 1000174c f   NativeCrypto.obj
 0001:0000078d       _Java_jdk_crypto_jniprovider_NativeCrypto_DigestReset@16 1000178d f   NativeCrypto.obj
 0001:000007e8       _Java_jdk_crypto_jniprovider_NativeCrypto_DigestUpdate@28 100017e8 f   NativeCrypto.obj
 0001:00000859       _Java_jdk_crypto_jniprovider_NativeCrypto_ECCreatePrivateKey@24 10001859 f   NativeCrypto.obj
 0001:000008c5       _Java_jdk_crypto_jniprovider_NativeCrypto_ECCreatePublicKey@36 100018c5 f   NativeCrypto.obj
 0001:00000996       _Java_jdk_crypto_jniprovider_NativeCrypto_ECDSASign@32 10001996 f   NativeCrypto.obj
 0001:00000a8c       _Java_jdk_crypto_jniprovider_NativeCrypto_ECDSAVerify@32 10001a8c f   NativeCrypto.obj
 0001:00000b7b       _Java_jdk_crypto_jniprovider_NativeCrypto_ECDeriveKey@36 10001b7b f   NativeCrypto.obj
 0001:00000be1       _Java_jdk_crypto_jniprovider_NativeCrypto_ECDestroyKey@16 10001be1 f   NativeCrypto.obj
 0001:00000bfd       _Java_jdk_crypto_jniprovider_NativeCrypto_ECEncodeGF@68 10001bfd f   NativeCrypto.obj
 0001:00000edd       _Java_jdk_crypto_jniprovider_NativeCrypto_ECGenerateKeyPair@44 10001edd f   NativeCrypto.obj
 0001:000010b1       _Java_jdk_crypto_jniprovider_NativeCrypto_ECNativeGF2m@8 100020b1 f   NativeCrypto.obj
 0001:000010b9       _Java_jdk_crypto_jniprovider_NativeCrypto_GCMDecrypt@72 100020b9 f   NativeCrypto.obj
 0001:0000132b       _Java_jdk_crypto_jniprovider_NativeCrypto_GCMEncrypt@72 1000232b f   NativeCrypto.obj
 0001:0000157e       _Java_jdk_crypto_jniprovider_NativeCrypto_PBEDerive@44 1000257e f   NativeCrypto.obj
 0001:00001698       _Java_jdk_crypto_jniprovider_NativeCrypto_PBKDF2Derive@28 10002698 f   NativeCrypto.obj
 0001:000017ef       _Java_jdk_crypto_jniprovider_NativeCrypto_RSADP@32 100027ef f   NativeCrypto.obj
 0001:00001954       _Java_jdk_crypto_jniprovider_NativeCrypto_RSAEP@28 10002954 f   NativeCrypto.obj
 0001:000019e0       _Java_jdk_crypto_jniprovider_NativeCrypto_createRSAPrivateCrtKey@72 100029e0 f   NativeCrypto.obj
 0001:00001ed7       _Java_jdk_crypto_jniprovider_NativeCrypto_createRSAPublicKey@24 10002ed7 f   NativeCrypto.obj
 0001:00001fb4       _Java_jdk_crypto_jniprovider_NativeCrypto_destroyRSAKey@16 10002fb4 f   NativeCrypto.obj
 0001:00001fc9       _Java_jdk_crypto_jniprovider_NativeCrypto_isMD5Available@8 10002fc9 f   NativeCrypto.obj
 0001:00001fd6       _Java_jdk_crypto_jniprovider_NativeCrypto_isOpenSSLFIPS@8 10002fd6 f   NativeCrypto.obj
 0001:00001fde       _Java_jdk_crypto_jniprovider_NativeCrypto_loadCrypto@24 10002fde f   NativeCrypto.obj
 0001:00002d88       _OSSL102_RSA_set0_crt_params 10003d88 f   NativeCrypto.obj
 0001:00002df9       _OSSL102_RSA_set0_factors  10003df9 f   NativeCrypto.obj
 0001:00002e49       _OSSL102_RSA_set0_key      10003e49 f   NativeCrypto.obj
 0001:00002eae       ___local_stdio_printf_options 10003eae f i NativeCrypto.obj
 0001:00002eb4       ___local_stdio_scanf_options 10003eb4 f i NativeCrypto.obj
 0001:00002eba       __vfprintf_l               10003eba f i NativeCrypto.obj
 0001:00002ede       __vsscanf_l                10003ede f i NativeCrypto.obj
 0001:00002f04       _convertJavaBItoBN         10003f04 f   NativeCrypto.obj
 0001:00003145       _fprintf                   10004145 f i NativeCrypto.obj
 0001:000034c7       _printf                    100044c7 f i NativeCrypto.obj
 0001:000034e5       _setECPublicCoordinates    100044e5 f   NativeCrypto.obj
 0001:000034fb       _setECPublicKey            100044fb f   NativeCrypto.obj
 0001:000035a6       _sscanf                    100045a6 f i NativeCrypto.obj
 0001:000036e6       @__security_check_cookie@4 100046e6 f   MSVCRT:secchk.obj
 0001:00003a34       __DllMainCRTStartup@12     10004a34 f   MSVCRT:dll_dllmain.obj
 0001:00003a57       ___raise_securityfailure   10004a57 f   MSVCRT:gs_report.obj
 0001:00003a7f       ___report_gsfailure        10004a7f f   MSVCRT:gs_report.obj
 0001:00003bc6       ___security_init_cookie    10004bc6 f   MSVCRT:gs_support.obj
 0001:00003c11       _DllMain@12                10004c11 f   MSVCRT:dll_dllmain_stub.obj
 0001:00003c33       ?__scrt_initialize_type_info@@YAXXZ 10004c33 f   MSVCRT:tncleanup.obj
 0001:00003c3f       ?__scrt_uninitialize_type_info@@YAXXZ 10004c3f f   MSVCRT:tncleanup.obj
 0001:00003c4b       ___scrt_initialize_default_local_stdio_options 10004c4b f   MSVCRT:default_local_stdio_options.obj
 0001:00003cac       ___scrt_acquire_startup_lock 10004cac f   MSVCRT:utility.obj
 0001:00003cde       ___scrt_dllmain_after_initialize_c 10004cde f   MSVCRT:utility.obj
 0001:00003d09       ___scrt_dllmain_before_initialize_c 10004d09 f   MSVCRT:utility.obj
 0001:00003d17       ___scrt_dllmain_crt_thread_attach 10004d17 f   MSVCRT:utility.obj
 0001:00003d36       ___scrt_dllmain_crt_thread_detach 10004d36 f   MSVCRT:utility.obj
 0001:00003d43       ___scrt_dllmain_exception_filter 10004d43 f   MSVCRT:utility.obj
 0001:00003d77       ___scrt_dllmain_uninitialize_c 10004d77 f   MSVCRT:utility.obj
 0001:00003d9a       ___scrt_dllmain_uninitialize_critical 10004d9a f   MSVCRT:utility.obj
 0001:00003da7       ___scrt_initialize_crt     10004da7 f   MSVCRT:utility.obj
 0001:00003de0       ___scrt_initialize_onexit_tables 10004de0 f   MSVCRT:utility.obj
 0001:00003e67       ___scrt_is_nonwritable_in_current_image 10004e67 f   MSVCRT:utility.obj
 0001:00003efb       ___scrt_release_startup_lock 10004efb f   MSVCRT:utility.obj
 0001:00003f18       ___scrt_uninitialize_crt   10004f18 f   MSVCRT:utility.obj
 0001:00003f40       ___scrt_get_dyn_tls_init_callback 10004f40 f   MSVCRT:dyn_tls_init.obj
 0001:00003f46       ___scrt_fastfail           10004f46 f   MSVCRT:utility_desktop.obj
 0001:00004061       __crt_debugger_hook        10005061 f   MSVCRT:utility_desktop.obj
 0001:00004069       __RTC_Initialize           10005069 f   MSVCRT:initsect.obj
 0001:00004095       __RTC_Terminate            10005095 f   MSVCRT:initsect.obj
 0001:000040d0       __SEH_prolog4              100050d0 f   MSVCRT:sehprolg4.obj
 0001:00004115       __except_handler4          10005115 f   MSVCRT:chandler4gs.obj
 0001:00004144       @_guard_check_icall_nop@4  10005144 f i MSVCRT:guard_support.obj
 0001:00004147       ___isa_available_init      10005147 f   MSVCRT:cpu_disp.obj
 0001:0000431b       __get_startup_argv_mode    1000531b f   MSVCRT:argv_mode.obj
 0001:0000431f       ___scrt_is_ucrt_dll_in_use 1000531f f   MSVCRT:ucrt_detection.obj
 0001:0000432b       _memset                    1000532b f   vcruntime:VCRUNTIME140.dll
 0001:00004331       ___std_type_info_destroy_list 10005331 f   vcruntime:VCRUNTIME140.dll
 0001:00004337       __except_handler4_common   10005337 f   vcruntime:VCRUNTIME140.dll
 0001:0000433d       _strcat                    1000533d f   ucrt:api-ms-win-crt-string-l1-1-0.dll
 0001:00004343       _strcpy                    10005343 f   ucrt:api-ms-win-crt-string-l1-1-0.dll
 0001:00004349       _strlen                    10005349 f   ucrt:api-ms-win-crt-string-l1-1-0.dll
 0001:0000434f       __initterm                 1000534f f   ucrt:api-ms-win-crt-runtime-l1-1-0.dll
 0001:00004355       __initterm_e               10005355 f   ucrt:api-ms-win-crt-runtime-l1-1-0.dll
 0001:0000435b       __seh_filter_dll           1000535b f   ucrt:api-ms-win-crt-runtime-l1-1-0.dll
 0001:00004361       __configure_narrow_argv    10005361 f   ucrt:api-ms-win-crt-runtime-l1-1-0.dll
 0001:00004367       __initialize_narrow_environment 10005367 f   ucrt:api-ms-win-crt-runtime-l1-1-0.dll
 0001:0000436d       __initialize_onexit_table  1000536d f   ucrt:api-ms-win-crt-runtime-l1-1-0.dll
 0001:00004373       __execute_onexit_table     10005373 f   ucrt:api-ms-win-crt-runtime-l1-1-0.dll
 0001:00004379       __cexit                    10005379 f   ucrt:api-ms-win-crt-runtime-l1-1-0.dll
 0001:0000437f       ___acrt_initialize         1000537f f   MSVCRT:ucrt_stubs.obj
 0001:0000437f       ___acrt_thread_attach      1000537f f   MSVCRT:ucrt_stubs.obj
 0001:0000437f       ___acrt_thread_detach      1000537f f   MSVCRT:ucrt_stubs.obj
 0001:0000437f       ___acrt_uninitialize       1000537f f   MSVCRT:ucrt_stubs.obj
 0001:0000437f       ___acrt_uninitialize_critical 1000537f f   MSVCRT:ucrt_stubs.obj
 0001:0000437f       ___scrt_stub_for_acrt_initialize 1000537f f   MSVCRT:ucrt_stubs.obj
 0001:0000437f       ___scrt_stub_for_acrt_thread_attach 1000537f f   MSVCRT:ucrt_stubs.obj
 0001:0000437f       ___scrt_stub_for_acrt_thread_detach 1000537f f   MSVCRT:ucrt_stubs.obj
 0001:0000437f       ___scrt_stub_for_acrt_uninitialize 1000537f f   MSVCRT:ucrt_stubs.obj
 0001:0000437f       ___scrt_stub_for_acrt_uninitialize_critical 1000537f f   MSVCRT:ucrt_stubs.obj
 0001:0000437f       ___vcrt_initialize         1000537f f   MSVCRT:ucrt_stubs.obj
 0001:0000437f       ___vcrt_thread_attach      1000537f f   MSVCRT:ucrt_stubs.obj
 0001:0000437f       ___vcrt_thread_detach      1000537f f   MSVCRT:ucrt_stubs.obj
 0001:0000437f       ___vcrt_uninitialize       1000537f f   MSVCRT:ucrt_stubs.obj
 0001:0000437f       ___vcrt_uninitialize_critical 1000537f f   MSVCRT:ucrt_stubs.obj
 0001:00004382       ___scrt_stub_for_is_c_termination_complete 10005382 f   MSVCRT:ucrt_stubs.obj
 0001:00004382       __is_c_termination_complete 10005382 f   MSVCRT:ucrt_stubs.obj
 0001:00004385       __filter_x86_sse2_floating_point_exception 10005385 f   MSVCRT:x86_exception_filter.obj
 0001:00004385       __filter_x86_sse2_floating_point_exception_default 10005385 f   MSVCRT:x86_exception_filter.obj
 0002:00000000       __imp__CloseHandle@4       10006000     kernel32:KERNEL32.dll
 0002:00000004       __imp__GetLastError@0      10006004     kernel32:KERNEL32.dll
 0002:00000008       __imp__ReleaseMutex@4      10006008     kernel32:KERNEL32.dll
 0002:0000000c       __imp__WaitForSingleObject@8 1000600c     kernel32:KERNEL32.dll
 0002:00000010       __imp__CreateMutexA@12     10006010     kernel32:KERNEL32.dll
 0002:00000014       __imp__FreeLibrary@4       10006014     kernel32:KERNEL32.dll
 0002:00000018       __imp__GetModuleFileNameA@12 10006018     kernel32:KERNEL32.dll
 0002:0000001c       __imp__GetProcAddress@8    1000601c     kernel32:KERNEL32.dll
 0002:00000020       __imp__LoadLibraryA@4      10006020     kernel32:KERNEL32.dll
 0002:00000024       __imp__LocalFree@4         10006024     kernel32:KERNEL32.dll
 0002:00000028       __imp__FormatMessageA@28   10006028     kernel32:KERNEL32.dll
 0002:0000002c       __imp__UnhandledExceptionFilter@4 1000602c     kernel32:KERNEL32.dll
 0002:00000030       __imp__SetUnhandledExceptionFilter@4 10006030     kernel32:KERNEL32.dll
 0002:00000034       __imp__GetCurrentProcess@0 10006034     kernel32:KERNEL32.dll
 0002:00000038       __imp__TerminateProcess@8  10006038     kernel32:KERNEL32.dll
 0002:0000003c       __imp__IsProcessorFeaturePresent@4 1000603c     kernel32:KERNEL32.dll
 0002:00000040       __imp__QueryPerformanceCounter@4 10006040     kernel32:KERNEL32.dll
 0002:00000044       __imp__GetCurrentProcessId@0 10006044     kernel32:KERNEL32.dll
 0002:00000048       __imp__GetCurrentThreadId@0 10006048     kernel32:KERNEL32.dll
 0002:0000004c       __imp__GetSystemTimeAsFileTime@4 1000604c     kernel32:KERNEL32.dll
 0002:00000050       __imp__DisableThreadLibraryCalls@4 10006050     kernel32:KERNEL32.dll
 0002:00000054       __imp__InitializeSListHead@4 10006054     kernel32:KERNEL32.dll
 0002:00000058       __imp__IsDebuggerPresent@0 10006058     kernel32:KERNEL32.dll
 0002:0000005c       \177KERNEL32_NULL_THUNK_DATA 1000605c     kernel32:KERNEL32.dll
 0002:00000060       __imp__memset              10006060     vcruntime:VCRUNTIME140.dll
 0002:00000064       __imp____std_type_info_destroy_list 10006064     vcruntime:VCRUNTIME140.dll
 0002:00000068       __imp___except_handler4_common 10006068     vcruntime:VCRUNTIME140.dll
 0002:0000006c       \177VCRUNTIME140_NULL_THUNK_DATA 1000606c     vcruntime:VCRUNTIME140.dll
 0002:00000070       __imp__free                10006070     ucrt:api-ms-win-crt-heap-l1-1-0.dll
 0002:00000074       __imp__malloc              10006074     ucrt:api-ms-win-crt-heap-l1-1-0.dll
 0002:00000078       \177api-ms-win-crt-heap-l1-1-0_NULL_THUNK_DATA 10006078     ucrt:api-ms-win-crt-heap-l1-1-0.dll
 0002:0000007c       __imp___initialize_onexit_table 1000607c     ucrt:api-ms-win-crt-runtime-l1-1-0.dll
 0002:00000080       __imp___initialize_narrow_environment 10006080     ucrt:api-ms-win-crt-runtime-l1-1-0.dll
 0002:00000084       __imp___cexit              10006084     ucrt:api-ms-win-crt-runtime-l1-1-0.dll
 0002:00000088       __imp___execute_onexit_table 10006088     ucrt:api-ms-win-crt-runtime-l1-1-0.dll
 0002:0000008c       __imp___initterm           1000608c     ucrt:api-ms-win-crt-runtime-l1-1-0.dll
 0002:00000090       __imp___initterm_e         10006090     ucrt:api-ms-win-crt-runtime-l1-1-0.dll
 0002:00000094       __imp___seh_filter_dll     10006094     ucrt:api-ms-win-crt-runtime-l1-1-0.dll
 0002:00000098       __imp___configure_narrow_argv 10006098     ucrt:api-ms-win-crt-runtime-l1-1-0.dll
 0002:0000009c       \177api-ms-win-crt-runtime-l1-1-0_NULL_THUNK_DATA 1000609c     ucrt:api-ms-win-crt-runtime-l1-1-0.dll
 0002:000000a0       __imp____stdio_common_vfprintf 100060a0     ucrt:api-ms-win-crt-stdio-l1-1-0.dll
 0002:000000a4       __imp__fflush              100060a4     ucrt:api-ms-win-crt-stdio-l1-1-0.dll
 0002:000000a8       __imp____acrt_iob_func     100060a8     ucrt:api-ms-win-crt-stdio-l1-1-0.dll
 0002:000000ac       __imp____stdio_common_vsscanf 100060ac     ucrt:api-ms-win-crt-stdio-l1-1-0.dll
 0002:000000b0       \177api-ms-win-crt-stdio-l1-1-0_NULL_THUNK_DATA 100060b0     ucrt:api-ms-win-crt-stdio-l1-1-0.dll
 0002:000000b4       __imp__tolower             100060b4     ucrt:api-ms-win-crt-string-l1-1-0.dll
 0002:000000b8       __imp__strcat              100060b8     ucrt:api-ms-win-crt-string-l1-1-0.dll
 0002:000000bc       __imp__strlen              100060bc     ucrt:api-ms-win-crt-string-l1-1-0.dll
 0002:000000c0       __imp__isalpha             100060c0     ucrt:api-ms-win-crt-string-l1-1-0.dll
 0002:000000c4       __imp__strcpy              100060c4     ucrt:api-ms-win-crt-string-l1-1-0.dll
 0002:000000c8       \177api-ms-win-crt-string-l1-1-0_NULL_THUNK_DATA 100060c8     ucrt:api-ms-win-crt-string-l1-1-0.dll
 0002:000000cc       ___guard_check_icall_fptr  100060cc     MSVCRT:guard_support.obj
 0002:000000d0       ___castguard_check_failure_os_handled_fptr 100060d0     MSVCRT:guard_support.obj
 0002:000000d4       ___xc_a                    100060d4     MSVCRT:initializers.obj
 0002:000000d8       ___xc_z                    100060d8     MSVCRT:initializers.obj
 0002:000000dc       ___xi_a                    100060dc     MSVCRT:initializers.obj
 0002:000000e0       ___xi_z                    100060e0     MSVCRT:initializers.obj
 0002:000000e4       ___xp_a                    100060e4     MSVCRT:initializers.obj
 0002:000000e8       ___xp_z                    100060e8     MSVCRT:initializers.obj
 0002:000000ec       ___xt_a                    100060ec     MSVCRT:initializers.obj
 0002:000000f0       ___xt_z                    100060f0     MSVCRT:initializers.obj
 0002:00000120       ??_C@_0BA@BGIGFJLH@libcrypto?93?4dll@ 10006120     NativeCrypto.obj
 0002:00000130       ??_C@_0BC@ICEILHCG@libcrypto?91_1?4dll@ 10006130     NativeCrypto.obj
 0002:00000144       ??_C@_0N@IEEBINGH@libeay32?4dll@ 10006144     NativeCrypto.obj
 0002:00000154       ??_C@_0BL@JFKAOCIF@An?5OpenSSL?5error?5occurred?6@ 10006154     NativeCrypto.obj
 0002:00000170       ??_C@_03OFAPEBGM@?$CFs?6@  10006170     NativeCrypto.obj
 0002:00000174       ??_C@_0BG@MBINOMKO@OpenSSL?5?$CFld?4?$CFld?4?$CFld?$CFc@ 10006174     NativeCrypto.obj
 0002:0000018c       ??_C@_0BO@FCDFIFHK@OpenSSL?5was?5loaded?5from?5?9?5?$CFs?6@ 1000618c     NativeCrypto.obj
 0002:000001ac       ??_C@_0BA@HPMBCNAB@OpenSSL_version@ 100061ac     NativeCrypto.obj
 0002:000001bc       ??_C@_0P@PIHLHJGN@SSLeay_version@ 100061bc     NativeCrypto.obj
 0002:000001d0       ??_C@_0FH@BAFCINAE@Error?5loading?5OpenSSL?3?5Error?5fi@ 100061d0     NativeCrypto.obj
 0002:00000228       ??_C@_0DP@JGPDADLC@Error?5loading?5OpenSSL?3?5Incompat@ 10006228     NativeCrypto.obj
 0002:00000268       ??_C@_0CH@LOBKHAIN@EVP_default_properties_is_fips_@ 10006268     NativeCrypto.obj
 0002:00000290       ??_C@_09BCJAEHEL@FIPS_mode@ 10006290     NativeCrypto.obj
 0002:0000029c       ??_C@_07KJFPOMFC@?$CFs?3?5?$CFs?6@ 1000629c     NativeCrypto.obj
 0002:000002a4       ??_C@_0BB@CMEKANCH@?$CIunknown?5reason?$CJ@ 100062a4     NativeCrypto.obj
 0002:000002b8       ??_C@_0BN@PCLDIFCP@Failed?5to?5load?5?$CFs?5due?5to?5?$CFs?6@ 100062b8     NativeCrypto.obj
 0002:000002d8       ??_C@_0DI@PFJKEFNN@Skipping?5trying?5to?5load?5a?5libra@ 100062d8     NativeCrypto.obj
 0002:00000310       ??_C@_0CG@LKMEGFEO@?7Failed?5to?5allocate?5memory?5for?5@ 10006310     NativeCrypto.obj
 0002:00000338       ??_C@_0DG@BHEPPKLO@Attempting?5to?5load?5library?5bund@ 10006338     NativeCrypto.obj
 0002:00000370       ??_C@_0BJ@IJGPDENH@?7Attempting?5to?5load?3?5?$CFs?6@ 10006370     NativeCrypto.obj
 0002:0000038c       ??_C@_0BJ@BOLPKGOH@?7?7Loaded?5OpenSSL?5version@ 1000638c     NativeCrypto.obj
 0002:000003a8       ??_C@_0CI@GFBPIMLI@Attempting?5to?5load?5libname?5from@ 100063a8     NativeCrypto.obj
 0002:000003d0       ??_C@_0BI@NNDBGBPB@?7Loaded?5OpenSSL?5version@ 100063d0     NativeCrypto.obj
 0002:000003e8       ??_C@_00CNPNBAHC@@         100063e8     NativeCrypto.obj
 0002:000003ec       ??_C@_0CN@KCODGBDO@Failed?5to?5get?5jdk?4native?4openss@ 100063ec     NativeCrypto.obj
 0002:0000041c       ??_C@_0DB@KNFOOGBB@The?5jdk?4native?4openssl?4lib?5prop@ 1000641c     NativeCrypto.obj
 0002:00000450       ??_C@_0EC@CELBJHCF@OpenSSL?5library?5specified?5in?5jd@ 10006450     NativeCrypto.obj
 0002:00000494       ??_C@_0CA@LGHBIFJG@Failed?5to?5get?5java?4home?5value?4?6@ 10006494     NativeCrypto.obj
 0002:000004b4       ??_C@_0CH@GMNJBKEN@FAILED?5TO?5LOAD?5OPENSSL?5CRYPTO?5L@ 100064b4     NativeCrypto.obj
 0002:000004dc       ??_C@_0CD@GMBNJAOJ@OpenSSL?5to?5be?5used?5was?5loaded?5f@ 100064dc     NativeCrypto.obj
 0002:00000500       ??_C@_0CI@NJCDBAGM@Version?5of?5OpenSSL?5library?5that@ 10006500     NativeCrypto.obj
 0002:00000528       ??_C@_0BD@KCMFIFPA@ERR_error_string_n@ 10006528     NativeCrypto.obj
 0002:0000053c       ??_C@_0BB@GICHBNCI@ERR_error_string@ 1000653c     NativeCrypto.obj
 0002:00000550       ??_C@_0O@CFFJHPAB@ERR_get_error@ 10006550     NativeCrypto.obj
 0002:00000560       ??_C@_0BB@COGJFOLI@CRYPTO_num_locks@ 10006560     NativeCrypto.obj
 0002:00000574       ??_C@_0BM@BPNHJJIG@CRYPTO_THREADID_set_numeric@ 10006574     NativeCrypto.obj
 0002:00000590       ??_C@_0O@JHFEPHEL@CRYPTO_malloc@ 10006590     NativeCrypto.obj
 0002:000005a0       ??_C@_0M@MLHDOKNM@CRYPTO_free@ 100065a0     NativeCrypto.obj
 0002:000005ac       ??_C@_0BN@KPFPHOHH@CRYPTO_THREADID_set_callback@ 100065ac     NativeCrypto.obj
 0002:000005cc       ??_C@_0BM@IOPFJNF@CRYPTO_set_locking_callback@ 100065cc     NativeCrypto.obj
 0002:000005e8       ??_C@_07CJMLOOOL@EVP_md5@  100065e8     NativeCrypto.obj
 0002:000005f0       ??_C@_08PBPOHJL@EVP_sha1@  100065f0     NativeCrypto.obj
 0002:000005fc       ??_C@_0L@BFNCDCPF@EVP_sha256@ 100065fc     NativeCrypto.obj
 0002:00000608       ??_C@_0L@CCKLEGPC@EVP_sha224@ 10006608     NativeCrypto.obj
 0002:00000614       ??_C@_0L@JHIAKEEB@EVP_sha384@ 10006614     NativeCrypto.obj
 0002:00000620       ??_C@_0L@OLGAGHJE@EVP_sha512@ 10006620     NativeCrypto.obj
 0002:0000062c       ??_C@_0P@FBDLFBDI@EVP_sha512_224@ 1000662c     NativeCrypto.obj
 0002:0000063c       ??_C@_0P@GGECCFDP@EVP_sha512_256@ 1000663c     NativeCrypto.obj
 0002:0000064c       ??_C@_0P@LBBHIKLM@EVP_MD_CTX_new@ 1000664c     NativeCrypto.obj
 0002:0000065c       ??_C@_0BB@LLCENKBD@EVP_MD_CTX_reset@ 1000665c     NativeCrypto.obj
 0002:00000670       ??_C@_0BA@DIPACEDG@EVP_MD_CTX_free@ 10006670     NativeCrypto.obj
 0002:00000680       ??_C@_0BC@CDDHKKMK@EVP_MD_CTX_create@ 10006680     NativeCrypto.obj
 0002:00000694       ??_C@_0BD@EAMOJGOK@EVP_MD_CTX_cleanup@ 10006694     NativeCrypto.obj
 0002:000006a8       ??_C@_0BD@HIKAFGJM@EVP_MD_CTX_destroy@ 100066a8     NativeCrypto.obj
 0002:000006bc       ??_C@_0BC@NBJFCNLO@EVP_DigestInit_ex@ 100066bc     NativeCrypto.obj
 0002:000006d0       ??_C@_0BD@OOMFHFKA@EVP_MD_CTX_copy_ex@ 100066d0     NativeCrypto.obj
 0002:000006e4       ??_C@_0BB@ECHJOJOG@EVP_DigestUpdate@ 100066e4     NativeCrypto.obj
 0002:000006f8       ??_C@_0BD@OFMHHJIG@EVP_DigestFinal_ex@ 100066f8     NativeCrypto.obj
 0002:0000070c       ??_C@_0BD@KDJHKKHN@EVP_CIPHER_CTX_new@ 1000670c     NativeCrypto.obj
 0002:00000720       ??_C@_0BE@NEIBFGDA@EVP_CIPHER_CTX_free@ 10006720     NativeCrypto.obj
 0002:00000734       ??_C@_0BA@MIPBGJPL@EVP_aes_128_cbc@ 10006734     NativeCrypto.obj
 0002:00000744       ??_C@_0BA@GLGNBOGH@EVP_aes_192_cbc@ 10006744     NativeCrypto.obj
 0002:00000754       ??_C@_0BA@LJNDDBOG@EVP_aes_256_cbc@ 10006754     NativeCrypto.obj
 0002:00000764       ??_C@_0BC@FOOGEGCP@EVP_CipherInit_ex@ 10006764     NativeCrypto.obj
 0002:00000778       ??_C@_0BL@GHJMPLKJ@EVP_CIPHER_CTX_set_padding@ 10006778     NativeCrypto.obj
 0002:00000794       ??_C@_0BB@FEIMIHDK@EVP_CipherUpdate@ 10006794     NativeCrypto.obj
 0002:000007a8       ??_C@_0BD@GCEAKJDP@EVP_CipherFinal_ex@ 100067a8     NativeCrypto.obj
 0002:000007bc       ??_C@_0BA@NINCLJBF@EVP_aes_128_gcm@ 100067bc     NativeCrypto.obj
 0002:000007cc       ??_C@_0BA@HLEOMOIJ@EVP_aes_192_gcm@ 100067cc     NativeCrypto.obj
 0002:000007dc       ??_C@_0BA@KJPAOBAI@EVP_aes_256_gcm@ 100067dc     NativeCrypto.obj
 0002:000007ec       ??_C@_0BE@PBKBIICA@EVP_CIPHER_CTX_ctrl@ 100067ec     NativeCrypto.obj
 0002:00000800       ??_C@_0BD@NJDNKKJM@EVP_DecryptInit_ex@ 10006800     NativeCrypto.obj
 0002:00000814       ??_C@_0BC@IHMDOGKL@EVP_DecryptUpdate@ 10006814     NativeCrypto.obj
 0002:00000828       ??_C@_0BB@PDIJBBLN@EVP_DecryptFinal@ 10006828     NativeCrypto.obj
 0002:0000083c       ??_C@_07BEDPMABO@RSA_new@  1000683c     NativeCrypto.obj
 0002:00000844       ??_C@_0N@CGJMOJGH@RSA_set0_key@ 10006844     NativeCrypto.obj
 0002:00000854       ??_C@_0BB@POEMEDBA@RSA_set0_factors@ 10006854     NativeCrypto.obj
 0002:00000868       ??_C@_0BE@IHFICCGA@RSA_set0_crt_params@ 10006868     NativeCrypto.obj
 0002:0000087c       ??_C@_08INMOLI@RSA_free@   1000687c     NativeCrypto.obj
 0002:00000888       ??_C@_0BD@PDPPPPCN@RSA_public_decrypt@ 10006888     NativeCrypto.obj
 0002:0000089c       ??_C@_0BE@GMELDCOG@RSA_private_decrypt@ 1000689c     NativeCrypto.obj
 0002:000008b0       ??_C@_06MLINBBBN@BN_new@   100068b0     NativeCrypto.obj
 0002:000008b8       ??_C@_09ODLDNKNE@BN_bin2bn@ 100068b8     NativeCrypto.obj
 0002:000008c4       ??_C@_0BA@NODPKDEN@BN_set_negative@ 100068c4     NativeCrypto.obj
 0002:000008d4       ??_C@_07JJFLCNND@BN_free@  100068d4     NativeCrypto.obj
 0002:000008dc       ??_C@_09MEANCIOF@BN_bn2bin@ 100068dc     NativeCrypto.obj
 0002:000008e8       ??_C@_0M@BMNNLAL@BN_num_bits@ 100068e8     NativeCrypto.obj
 0002:000008f4       ??_C@_0BE@MFFKFHAB@EC_KEY_generate_key@ 100068f4     NativeCrypto.obj
 0002:00000908       ??_C@_0M@NMKCGAJN@EC_KEY_free@ 10006908     NativeCrypto.obj
 0002:00000914       ??_C@_0BB@IOKCFGPF@ECDH_compute_key@ 10006914     NativeCrypto.obj
 0002:00000928       ??_C@_0BH@OFCAHLIM@EC_KEY_get0_public_key@ 10006928     NativeCrypto.obj
 0002:00000940       ??_C@_0BI@IHBMKFAL@EC_KEY_get0_private_key@ 10006940     NativeCrypto.obj
 0002:00000958       ??_C@_0L@ONJMCKDA@EC_KEY_new@ 10006958     NativeCrypto.obj
 0002:00000964       ??_C@_0CJ@PKPNGFF@EC_KEY_set_public_key_affine_co@ 10006964     NativeCrypto.obj
 0002:00000990       ??_C@_0BH@ELJHICGP@EC_KEY_set_private_key@ 10006990     NativeCrypto.obj
 0002:000009a8       ??_C@_0L@OIEJOLGJ@BN_CTX_new@ 100069a8     NativeCrypto.obj
 0002:000009b4       ??_C@_0BH@LMGLLNHD@EC_GROUP_new_curve_GFp@ 100069b4     NativeCrypto.obj
 0002:000009cc       ??_C@_0BI@GKPNAHHP@EC_GROUP_new_curve_GF2m@ 100069cc     NativeCrypto.obj
 0002:000009e4       ??_C@_0BB@NIEGABFH@EC_KEY_set_group@ 100069e4     NativeCrypto.obj
 0002:000009f8       ??_C@_0N@LOIMDOGK@EC_POINT_new@ 100069f8     NativeCrypto.obj
 0002:00000a08       ??_C@_0BH@CFECBPOO@EC_GROUP_set_generator@ 10006a08     NativeCrypto.obj
 0002:00000a20       ??_C@_0BC@KEIEKAMA@EC_KEY_get0_group@ 10006a20     NativeCrypto.obj
 0002:00000a34       ??_C@_0O@FHEPMIGD@EC_POINT_free@ 10006a34     NativeCrypto.obj
 0002:00000a44       ??_C@_0O@KEFGGDJH@EC_GROUP_free@ 10006a44     NativeCrypto.obj
 0002:00000a54       ??_C@_0M@MOBAFMAM@BN_CTX_free@ 10006a54     NativeCrypto.obj
 0002:00000a60       ??_C@_0BG@GCHAIKDI@EC_KEY_set_public_key@ 10006a60     NativeCrypto.obj
 0002:00000a78       ??_C@_0BB@NNGADNNL@EC_KEY_check_key@ 10006a78     NativeCrypto.obj
 0002:00000a8c       ??_C@_0CA@GKCLEFHF@EC_POINT_set_affine_coordinates@ 10006a8c     NativeCrypto.obj
 0002:00000aac       ??_C@_0CA@GLAFGCKK@EC_POINT_get_affine_coordinates@ 10006aac     NativeCrypto.obj
 0002:00000acc       ??_C@_0CE@BGAPNKLA@EC_POINT_set_affine_coordinates@ 10006acc     NativeCrypto.obj
 0002:00000af0       ??_C@_0CF@GIDKPABC@EC_POINT_set_affine_coordinates@ 10006af0     NativeCrypto.obj
 0002:00000b18       ??_C@_0CE@CJDKBKKA@EC_POINT_get_affine_coordinates@ 10006b18     NativeCrypto.obj
 0002:00000b3c       ??_C@_0CF@HFLCNFLG@EC_POINT_get_affine_coordinates@ 10006b3c     NativeCrypto.obj
 0002:00000b64       ??_C@_0O@HPIOKGCH@ECDSA_do_sign@ 10006b64     NativeCrypto.obj
 0002:00000b74       ??_C@_0BA@EHPKHBIM@ECDSA_do_verify@ 10006b74     NativeCrypto.obj
 0002:00000b84       ??_C@_0O@LCAMPHNJ@ECDSA_SIG_new@ 10006b84     NativeCrypto.obj
 0002:00000b94       ??_C@_0P@FCLKKJM@ECDSA_SIG_free@ 10006b94     NativeCrypto.obj
 0002:00000ba4       ??_C@_0BB@IIOJIAAH@ECDSA_SIG_get0_r@ 10006ba4     NativeCrypto.obj
 0002:00000bb8       ??_C@_0BB@JBPCLBEG@ECDSA_SIG_get0_s@ 10006bb8     NativeCrypto.obj
 0002:00000bcc       ??_C@_0P@LKMNLNBO@ECDSA_SIG_set0@ 10006bcc     NativeCrypto.obj
 0002:00000bdc       ??_C@_0BD@DMMKPAAN@PKCS12_key_gen_uni@ 10006bdc     NativeCrypto.obj
 0002:00000bf0       ??_C@_0BC@KMIHJAOO@PKCS5_PBKDF2_HMAC@ 10006bf0     NativeCrypto.obj
 0002:00000c08       ??_C@_0EI@MPDAOHNE@Error?5loading?5OpenSSL?3?5One?5or?5m@ 10006c08     NativeCrypto.obj
 0002:00000c50       ??_C@_0DG@CJHOCNOH@Error?5loading?5OpenSSL?3?5Thread?5s@ 10006c50     NativeCrypto.obj
 0002:00000c88       ??_C@_0CG@HPEIDEDC@OpenSSL?5library?5loaded?5successf@ 10006c88     NativeCrypto.obj
 0002:00000cb0       ??_C@_0BH@KCAMECBI@CreateMutex?5error?3?5?$CFd?6@ 10006cb0     NativeCrypto.obj
 0002:00000cc8       ??_C@_0BH@FPGCIENB@CloseHandle?5error?3?5?$CFd?6@ 10006cc8     NativeCrypto.obj
 0002:00000ce0       ??_C@_0BP@OBCPLEDE@WaitForSingleObject?5error?3?5?$CFd?6@ 10006ce0     NativeCrypto.obj
 0002:00000d00       ??_C@_0BI@DELFCGJD@ReleaseMutex?5error?3?5?$CFd?6@ 10006d00     NativeCrypto.obj
 0002:00000d18       ??_C@_0BJ@LFBOMBKK@destoryResult?5error?3?5?$CFd?6@ 10006d18     NativeCrypto.obj
 0002:00000d34       ??_C@_0CG@LFHDDGAP@Failed?5to?5create?5an?5ECDSA?5Signa@ 10006d34     NativeCrypto.obj
 0002:00000d5c       __pDefaultRawDllMain       10006d5c     MSVCRT:dll_dllmain.obj
 0002:00000d5c       __pRawDllMain              10006d5c     MSVCRT:dll_dllmain.obj
 0002:00000d68       __load_config_used         10006d68     MSVCRT:loadcfg.obj
 0002:00000e80       ___safe_se_handler_table   10006e80     <linker-defined>
 0002:00000e84       ___volatile_metadata       10006e84     <linker-defined>
 0002:000011d4       ___rtc_iaa                 100071d4     MSVCRT:initsect.obj
 0002:000011d8       ___rtc_izz                 100071d8     MSVCRT:initsect.obj
 0002:000011dc       ___rtc_taa                 100071dc     MSVCRT:initsect.obj
 0002:000011e0       ___rtc_tzz                 100071e0     MSVCRT:initsect.obj
 0002:00001b14       __IMPORT_DESCRIPTOR_KERNEL32 10007b14     kernel32:KERNEL32.dll
 0002:00001b28       __IMPORT_DESCRIPTOR_VCRUNTIME140 10007b28     vcruntime:VCRUNTIME140.dll
 0002:00001b3c       __IMPORT_DESCRIPTOR_api-ms-win-crt-string-l1-1-0 10007b3c     ucrt:api-ms-win-crt-string-l1-1-0.dll
 0002:00001b50       __IMPORT_DESCRIPTOR_api-ms-win-crt-stdio-l1-1-0 10007b50     ucrt:api-ms-win-crt-stdio-l1-1-0.dll
 0002:00001b64       __IMPORT_DESCRIPTOR_api-ms-win-crt-heap-l1-1-0 10007b64     ucrt:api-ms-win-crt-heap-l1-1-0.dll
 0002:00001b78       __IMPORT_DESCRIPTOR_api-ms-win-crt-runtime-l1-1-0 10007b78     ucrt:api-ms-win-crt-runtime-l1-1-0.dll
 0002:00001b8c       __NULL_IMPORT_DESCRIPTOR   10007b8c     kernel32:KERNEL32.dll
 0003:00000000       ___security_cookie_complement 10009000     MSVCRT:gs_cookie.obj
 0003:00000004       ___security_cookie         10009004     MSVCRT:gs_cookie.obj
 0003:00000008       ___scrt_native_dllmain_reason 10009008     MSVCRT:utility.obj
 0003:00000010       ___isa_enabled             10009010     MSVCRT:cpu_disp.obj
 0003:00000014       ___scrt_ucrt_dll_is_in_use 10009014     MSVCRT:ucrt_stubs.obj
 0003:00000018       _first_time_gcm            10009018     NativeCrypto.obj
 0003:00000368       ?__type_info_root_node@@3U__type_info_node@@A 10009368     MSVCRT:tncleanup.obj
 0003:00000370       ___scrt_current_native_startup_state 10009370     MSVCRT:utility.obj
 0003:00000374       ___scrt_native_startup_lock 10009374     MSVCRT:utility.obj
 0003:00000394       ___scrt_debugger_hook_flag 10009394     MSVCRT:utility_desktop.obj
 0003:00000398       ___isa_available           10009398     MSVCRT:cpu_disp.obj
 0003:0000039c       ___favor                   1000939c     MSVCRT:cpu_disp.obj
 0003:000003a0       ?_OptionsStorage@?1??__local_stdio_scanf_options@@9@9 100093a0     <common>
 0003:000003a8       ?_OptionsStorage@?1??__local_stdio_printf_options@@9@9 100093a8     <common>
 0003:000003b0       _OSSL_PKCS5_PBKDF2_HMAC    100093b0     <common>
 0003:000003b4       _OSSL_PKCS12_key_gen       100093b4     <common>
 0003:000003b8       _OSSL_ECDSA_SIG_set0       100093b8     <common>
 0003:000003bc       _OSSL_ECDSA_SIG_get0_s     100093bc     <common>
 0003:000003c0       _OSSL_ECDSA_SIG_get0_r     100093c0     <common>
 0003:000003c4       _OSSL_ECDSA_SIG_free       100093c4     <common>
 0003:000003c8       _OSSL_ECDSA_SIG_new        100093c8     <common>
 0003:000003cc       _OSSL_ECDSA_do_verify      100093cc     <common>
 0003:000003d0       _OSSL_ECDSA_do_sign        100093d0     <common>
 0003:000003d4       _OSSL_EC_KEY_get0_private_key 100093d4     <common>
 0003:000003d8       _EC_set_public_key         100093d8     <common>
 0003:000003dc       _OSSL_EC_KEY_check_key     100093dc     <common>
 0003:000003e0       _OSSL_EC_KEY_set_public_key 100093e0     <common>
 0003:000003e4       _OSSL_BN_CTX_free          100093e4     <common>
 0003:000003e8       _OSSL_EC_GROUP_free        100093e8     <common>
 0003:000003ec       _OSSL_EC_POINT_free        100093ec     <common>
 0003:000003f0       _OSSL_EC_KEY_get0_group    100093f0     <common>
 0003:000003f4       _OSSL_EC_GROUP_set_generator 100093f4     <common>
 0003:000003f8       _OSSL_EC_POINT_get_affine_coordinates_GF2m 100093f8     <common>
 0003:000003fc       _OSSL_EC_POINT_get_affine_coordinates_GFp 100093fc     <common>
 0003:00000400       _OSSL_EC_POINT_set_affine_coordinates_GF2m 10009400     <common>
 0003:00000404       _OSSL_EC_POINT_set_affine_coordinates_GFp 10009404     <common>
 0003:00000408       _OSSL_EC_POINT_new         10009408     <common>
 0003:0000040c       _OSSL_EC_KEY_set_group     1000940c     <common>
 0003:00000410       _OSSL_EC_GROUP_new_curve_GF2m 10009410     <common>
 0003:00000414       _OSSL_EC_GROUP_new_curve_GFp 10009414     <common>
 0003:00000418       _OSSL_BN_CTX_new           10009418     <common>
 0003:0000041c       _OSSL_EC_KEY_set_private_key 1000941c     <common>
 0003:00000420       _OSSL_EC_KEY_set_public_key_affine_coordinates 10009420     <common>
 0003:00000424       _OSSL_EC_KEY_new           10009424     <common>
 0003:00000428       _OSSL_EC_KEY_get0_public_key 10009428     <common>
 0003:0000042c       _OSSL_ECDH_compute_key     1000942c     <common>
 0003:00000430       _OSSL_EC_KEY_free          10009430     <common>
 0003:00000434       _OSSL_EC_KEY_generate_key  10009434     <common>
 0003:00000438       _OSSL_BN_num_bits          10009438     <common>
 0003:0000043c       _OSSL_BN_bn2bin            1000943c     <common>
 0003:00000440       _OSSL_BN_free              10009440     <common>
 0003:00000444       _OSSL_BN_set_negative      10009444     <common>
 0003:00000448       _OSSL_BN_bin2bn            10009448     <common>
 0003:0000044c       _OSSL_BN_new               1000944c     <common>
 0003:00000450       _OSSL_RSA_private_encrypt  10009450     <common>
 0003:00000454       _OSSL_RSA_public_decrypt   10009454     <common>
 0003:00000458       _OSSL_RSA_free             10009458     <common>
 0003:0000045c       _OSSL_RSA_set0_crt_params  1000945c     <common>
 0003:00000460       _OSSL_RSA_set0_factors     10009460     <common>
 0003:00000464       _OSSL_RSA_set0_key         10009464     <common>
 0003:00000468       _OSSL_RSA_new              10009468     <common>
 0003:0000046c       _OSSL_DecryptFinal         1000946c     <common>
 0003:00000470       _OSSL_DecryptUpdate        10009470     <common>
 0003:00000474       _OSSL_DecryptInit_ex       10009474     <common>
 0003:00000478       _OSSL_CIPHER_CTX_ctrl      10009478     <common>
 0003:0000047c       _OSSL_aes_256_gcm          1000947c     <common>
 0003:00000480       _OSSL_aes_192_gcm          10009480     <common>
 0003:00000484       _OSSL_aes_128_gcm          10009484     <common>
 0003:00000488       _OSSL_CipherFinal_ex       10009488     <common>
 0003:0000048c       _OSSL_CipherUpdate         1000948c     <common>
 0003:00000490       _OSSL_CIPHER_CTX_set_padding 10009490     <common>
 0003:00000494       _OSSL_CipherInit_ex        10009494     <common>
 0003:00000498       _OSSL_aes_256_cbc          10009498     <common>
 0003:0000049c       _OSSL_aes_192_cbc          1000949c     <common>
 0003:000004a0       _OSSL_aes_128_cbc          100094a0     <common>
 0003:000004a4       _OSSL_CIPHER_CTX_free      100094a4     <common>
 0003:000004a8       _OSSL_CIPHER_CTX_new       100094a8     <common>
 0003:000004ac       _OSSL_MD_CTX_free          100094ac     <common>
 0003:000004b0       _OSSL_MD_CTX_reset         100094b0     <common>
 0003:000004b4       _OSSL_DigestFinal_ex       100094b4     <common>
 0003:000004b8       _OSSL_DigestUpdate         100094b8     <common>
 0003:000004bc       _OSSL_MD_CTX_copy_ex       100094bc     <common>
 0003:000004c0       _OSSL_DigestInit_ex        100094c0     <common>
 0003:000004c4       _OSSL_MD_CTX_new           100094c4     <common>
 0003:000004c8       _OSSL_sha512_256           100094c8     <common>
 0003:000004cc       _OSSL_sha512_224           100094cc     <common>
 0003:000004d0       _OSSL_sha512               100094d0     <common>
 0003:000004d4       _OSSL_sha384               100094d4     <common>
 0003:000004d8       _OSSL_sha224               100094d8     <common>
 0003:000004dc       _OSSL_sha256               100094dc     <common>
 0003:000004e0       _OSSL_sha1                 100094e0     <common>
 0003:000004e4       _OSSL_md5                  100094e4     <common>
 0003:000004e8       _OSSL_get_error            100094e8     <common>
 0003:000004ec       _OSSL_error_string         100094ec     <common>
 0003:000004f0       _OSSL_error_string_n       100094f0     <common>
 0003:000004f4       _OSSL_ECGF2M               100094f4     <common>
 0003:000004f8       ___dyn_tls_init_callback   100094f8     <common>

 entry point at        0001:00003a34

 Static symbols

 0000:ffff4000       .debug$S                   10000000     jncrypto.exp
 0000:ffff4000       .debug$S                   10000000     vcruntime:VCRUNTIME140.dll
 0000:ffff4000       .debug$S                   10000000     vcruntime:VCRUNTIME140.dll
 0000:ffff4000       .debug$S                   10000000     vcruntime:VCRUNTIME140.dll
 0000:ffff4000       .debug$S                   10000000     vcruntime:VCRUNTIME140.dll
 0000:ffff4000       .debug$S                   10000000     vcruntime:VCRUNTIME140.dll
 0000:ffff4000       .debug$S                   10000000     ucrt:api-ms-win-crt-heap-l1-1-0.dll
 0000:ffff4000       .debug$S                   10000000     ucrt:api-ms-win-crt-heap-l1-1-0.dll
 0000:ffff4000       .debug$S                   10000000     ucrt:api-ms-win-crt-runtime-l1-1-0.dll
 0000:ffff4000       .debug$S                   10000000     ucrt:api-ms-win-crt-runtime-l1-1-0.dll
 0000:ffff4000       .debug$S                   10000000     ucrt:api-ms-win-crt-runtime-l1-1-0.dll
 0000:ffff4000       .debug$S                   10000000     ucrt:api-ms-win-crt-runtime-l1-1-0.dll
 0000:ffff4000       .debug$S                   10000000     ucrt:api-ms-win-crt-runtime-l1-1-0.dll
 0000:ffff4000       .debug$S                   10000000     ucrt:api-ms-win-crt-runtime-l1-1-0.dll
 0000:ffff4000       .debug$S                   10000000     ucrt:api-ms-win-crt-runtime-l1-1-0.dll
 0000:ffff4000       .debug$S                   10000000     ucrt:api-ms-win-crt-runtime-l1-1-0.dll
 0000:ffff4000       .debug$S                   10000000     ucrt:api-ms-win-crt-runtime-l1-1-0.dll
 0000:ffff4000       .debug$S                   10000000     ucrt:api-ms-win-crt-runtime-l1-1-0.dll
 0000:ffff4000       .debug$S                   10000000     ucrt:api-ms-win-crt-runtime-l1-1-0.dll
 0000:ffff4000       .debug$S                   10000000     ucrt:api-ms-win-crt-runtime-l1-1-0.dll
 0000:ffff4000       .debug$S                   10000000     ucrt:api-ms-win-crt-stdio-l1-1-0.dll
 0000:ffff4000       .debug$S                   10000000     ucrt:api-ms-win-crt-stdio-l1-1-0.dll
 0000:ffff4000       .debug$S                   10000000     ucrt:api-ms-win-crt-stdio-l1-1-0.dll
 0000:ffff4000       .debug$S                   10000000     ucrt:api-ms-win-crt-stdio-l1-1-0.dll
 0000:ffff4000       .debug$S                   10000000     ucrt:api-ms-win-crt-string-l1-1-0.dll
 0000:ffff4000       .debug$S                   10000000     ucrt:api-ms-win-crt-string-l1-1-0.dll
 0000:ffff4000       .debug$S                   10000000     ucrt:api-ms-win-crt-string-l1-1-0.dll
 0000:ffff4000       .debug$S                   10000000     ucrt:api-ms-win-crt-string-l1-1-0.dll
 0000:ffff4000       .debug$S                   10000000     ucrt:api-ms-win-crt-string-l1-1-0.dll
 0000:ffff4000       .debug$S                   10000000     kernel32:KERNEL32.dll
 0000:ffff4000       .debug$S                   10000000     kernel32:KERNEL32.dll
 0000:ffff4000       .debug$S                   10000000     kernel32:KERNEL32.dll
 0000:ffff4000       .debug$S                   10000000     kernel32:KERNEL32.dll
 0000:ffff4000       .debug$S                   10000000     kernel32:KERNEL32.dll
 0000:ffff4000       .debug$S                   10000000     kernel32:KERNEL32.dll
 0000:ffff4000       .debug$S                   10000000     kernel32:KERNEL32.dll
 0000:ffff4000       .debug$S                   10000000     kernel32:KERNEL32.dll
 0000:ffff4000       .debug$S                   10000000     kernel32:KERNEL32.dll
 0000:ffff4000       .debug$S                   10000000     kernel32:KERNEL32.dll
 0000:ffff4000       .debug$S                   10000000     kernel32:KERNEL32.dll
 0000:ffff4000       .debug$S                   10000000     kernel32:KERNEL32.dll
 0000:ffff4000       .debug$S                   10000000     kernel32:KERNEL32.dll
 0000:ffff4000       .debug$S                   10000000     kernel32:KERNEL32.dll
 0000:ffff4000       .debug$S                   10000000     kernel32:KERNEL32.dll
 0000:ffff4000       .debug$S                   10000000     kernel32:KERNEL32.dll
 0000:ffff4000       .debug$S                   10000000     kernel32:KERNEL32.dll
 0000:ffff4000       .debug$S                   10000000     kernel32:KERNEL32.dll
 0000:ffff4000       .debug$S                   10000000     kernel32:KERNEL32.dll
 0000:ffff4000       .debug$S                   10000000     kernel32:KERNEL32.dll
 0000:ffff4000       .debug$S                   10000000     kernel32:KERNEL32.dll
 0000:ffff4000       .debug$S                   10000000     kernel32:KERNEL32.dll
 0000:ffff4000       .debug$S                   10000000     kernel32:KERNEL32.dll
 0000:ffff4000       .debug$S                   10000000     kernel32:KERNEL32.dll
 0000:ffff4000       .debug$S                   10000000     kernel32:KERNEL32.dll
 0001:00000000       _ECEncodeGF2m              10001000 f   NativeCrypto.obj
 0001:000000bf       _ECEncodeGFp               100010bf f   NativeCrypto.obj
 0001:0000072c       $LN22                      1000172c     NativeCrypto.obj
 0001:00002f64       _extractVersionToJlong     10003f64 f   NativeCrypto.obj
 0001:00002feb       _find_crypto_library       10003feb f   NativeCrypto.obj
 0001:0000315d       _getArrayFromBN            1000415d f   NativeCrypto.obj
 0001:000031b5       _get_crypto_library_version 100041b5 f   NativeCrypto.obj
 0001:0000335f       _load_crypto_library       1000435f f   NativeCrypto.obj
 0001:000033e1       _log_crypto_library_path   100043e1 f   NativeCrypto.obj
 0001:00003451       _printErrors               10004451 f   NativeCrypto.obj
 0001:000035be       _thread_setup              100045be f   NativeCrypto.obj
 0001:00003689       _win32_locking_callback    10004689 f   NativeCrypto.obj
 0001:000036f4       ?dllmain_crt_dispatch@@YGHQAUHINSTANCE__@@KQAX@Z 100046f4 f   MSVCRT:dll_dllmain.obj
 0001:00003747       ?dllmain_crt_process_attach@@YAHQAUHINSTANCE__@@QAX@Z 10004747 f   MSVCRT:dll_dllmain.obj
 0001:0000384e       ?dllmain_crt_process_detach@@YAH_N@Z 1000484e f   MSVCRT:dll_dllmain.obj
 0001:000038fe       ?dllmain_dispatch@@YAHQAUHINSTANCE__@@KQAX@Z 100048fe f   MSVCRT:dll_dllmain.obj
 0001:00003a09       ?dllmain_raw@@YGHQAUHINSTANCE__@@KQAX@Z 10004a09 f   MSVCRT:dll_dllmain.obj
 0001:00003b79       ___get_entropy             10004b79 f   MSVCRT:gs_support.obj
 0001:00003c68       ?find_pe_section@@YAPAU_IMAGE_SECTION_HEADER@@QAEI@Z 10004c68 f   MSVCRT:utility.obj
 0001:000040d0       $$000000                   100050d0     MSVCRT:sehprolg4.obj
 0002:000000f8       ?libNames@?1??find_crypto_library@@9@9 100060f8     NativeCrypto.obj
 0002:00000104       ?bundledLibName@?1??find_crypto_library@@9@9 10006104     NativeCrypto.obj
 0002:00000118       ?pathSuffix@?5??find_crypto_library@@9@9 10006118     NativeCrypto.obj
 0002:00000d60       _GS_ExceptionPointers      10006d60     MSVCRT:gs_report.obj
 0002:000011e8       __sehtable$?dllmain_crt_process_attach@@YAHQAUHINSTANCE__@@QAX@Z 100071e8     MSVCRT:dll_dllmain.obj
 0002:00001208       __sehtable$?dllmain_crt_process_detach@@YAH_N@Z 10007208     MSVCRT:dll_dllmain.obj
 0002:00001230       __sehtable$?dllmain_dispatch@@YAHQAUHINSTANCE__@@KQAX@Z 10007230     MSVCRT:dll_dllmain.obj
 0002:00001250       __sehtable$___scrt_is_nonwritable_in_current_image 10007250     MSVCRT:utility.obj
 0002:00001270       .edata                     10007270     jncrypto.exp
 0002:00001298       rgpv                       10007298     jncrypto.exp
 0002:00001318       rgszName                   10007318     jncrypto.exp
 0002:00001398       rgwOrd                     10007398     jncrypto.exp
 0002:000013d8       szName                     100073d8     jncrypto.exp
 0002:000013e5       $N00001                    100073e5     jncrypto.exp
 0002:000013f5       $N00002                    100073f5     jncrypto.exp
 0002:00001432       $N00003                    10007432     jncrypto.exp
 0002:00001467       $N00004                    10007467     jncrypto.exp
 0002:0000149e       $N00005                    1000749e     jncrypto.exp
 0002:000014d8       $N00006                    100074d8     jncrypto.exp
 0002:00001514       $N00007                    10007514     jncrypto.exp
 0002:00001557       $N00008                    10007557     jncrypto.exp
 0002:00001598       $N00009                    10007598     jncrypto.exp
 0002:000015da       $N00010                    100075da     jncrypto.exp
 0002:00001613       $N00011                    10007613     jncrypto.exp
 0002:0000164d       $N00012                    1000764d     jncrypto.exp
 0002:0000168d       $N00013                    1000768d     jncrypto.exp
 0002:000016cc       $N00014                    100076cc     jncrypto.exp
 0002:00001703       $N00015                    10007703     jncrypto.exp
 0002:0000173c       $N00016                    1000773c     jncrypto.exp
 0002:00001775       $N00017                    10007775     jncrypto.exp
 0002:000017af       $N00018                    100077af     jncrypto.exp
 0002:000017e7       $N00019                    100077e7     jncrypto.exp
 0002:00001826       $N00020                    10007826     jncrypto.exp
 0002:0000185f       $N00021                    1000785f     jncrypto.exp
 0002:00001897       $N00022                    10007897     jncrypto.exp
 0002:000018cf       $N00023                    100078cf     jncrypto.exp
 0002:00001906       $N00024                    10007906     jncrypto.exp
 0002:00001940       $N00025                    10007940     jncrypto.exp
 0002:00001973       $N00026                    10007973     jncrypto.exp
 0002:000019a6       $N00027                    100079a6     jncrypto.exp
 0002:000019ea       $N00028                    100079ea     jncrypto.exp
 0002:00001a2a       $N00029                    10007a2a     jncrypto.exp
 0002:00001a65       $N00030                    10007a65     jncrypto.exp
 0002:00001aa0       $N00031                    10007aa0     jncrypto.exp
 0002:00001ada       $N00032                    10007ada     jncrypto.exp
 0002:00001e48       .idata$6                   10007e48     kernel32:KERNEL32.dll
 0002:00001e9a       .idata$6                   10007e9a     vcruntime:VCRUNTIME140.dll
 0002:00001fe6       .idata$6                   10007fe6     ucrt:api-ms-win-crt-string-l1-1-0.dll
 0002:00002008       .idata$6                   10008008     ucrt:api-ms-win-crt-stdio-l1-1-0.dll
 0002:00002028       .idata$6                   10008028     ucrt:api-ms-win-crt-heap-l1-1-0.dll
 0002:00002048       .idata$6                   10008048     ucrt:api-ms-win-crt-runtime-l1-1-0.dll
 0003:0000001c       _OSSL_IS_FIPS              1000901c     NativeCrypto.obj
 0003:00000020       _OSSL_CRYPTO_num_locks     10009020     NativeCrypto.obj
 0003:00000024       _OSSL_CRYPTO_THREADID_set_numeric 10009024     NativeCrypto.obj
 0003:00000028       _OSSL_OPENSSL_malloc       10009028     NativeCrypto.obj
 0003:0000002c       _OSSL_OPENSSL_free         1000902c     NativeCrypto.obj
 0003:00000030       _OSSL_CRYPTO_THREADID_set_callback 10009030     NativeCrypto.obj
 0003:00000034       _OSSL_CRYPTO_set_locking_callback 10009034     NativeCrypto.obj
 0003:00000038       _crypto_library            10009038     NativeCrypto.obj
 0003:0000003c       _lock_cs                   1000903c     NativeCrypto.obj
 0003:00000040       ?__proc_attached@@3HA      10009040     MSVCRT:dll_dllmain.obj
 0003:00000048       _GS_ExceptionRecord        10009048     MSVCRT:gs_report.obj
 0003:00000098       _GS_ContextRecord          10009098     MSVCRT:gs_report.obj
 0003:00000378       ?is_initialized_as_dll@@3_NA 10009378     MSVCRT:utility.obj
 0003:00000379       ?module_local_atexit_table_initialized@@3_NA 10009379     MSVCRT:utility.obj
 0003:0000037c       ?module_local_atexit_table@@3U_onexit_table_t@@A 1000937c     MSVCRT:utility.obj
 0003:00000388       ?module_local_at_quick_exit_table@@3U_onexit_table_t@@A 10009388     MSVCRT:utility.obj
 0004:00000060       $R000000                   1000a060     jncrypto.dll.res
